:020000040000FA
:04080000E4EF07F02A
:1008100003B210EF05F0F2B42BEF05F09EB033EF0A
:1008200005F09EB23BEF05F0F2A81AEF04F0F2B229
:1008300025EF04F0F2A620EF04F0F2B022EF04F06E
:1008400093EF07F0F296F290FF00CD90F2929EA007
:100850002FEF04F00101533F2FEF04F0542BAEC1F2
:10086000B2F1AFC1B3F1B0C1B4F1B1C1B5F1AAC138
:10087000AEF1ABC1AFF1ACC1B0F1ADC1B1F1A6C148
:10088000AAF1A7C1ABF1A8C1ACF1A9C1ADF1A2C158
:10089000A6F1A3C1A7F1A4C1A8F1A5C1A9F19EC168
:1008A000A2F19FC1A3F1A0C1A4F1A1C1A5F19AC178
:1008B0009EF19BC19FF19CC1A0F19DC1A1F196C188
:1008C0009AF197C19BF198C19CF199C19DF1CECF4E
:1008D00096F1CFCF97F153C198F154C199F1CF6AF6
:1008E000CE6A0101536B546B9E90CD800FBC0F8E6E
:1008F0000FBA7EEF04F00F8A93EF07F00F8C0FBE54
:10090000BAEF04F096C19AF197C19BF198C19CF19E
:1009100099C19DF19AC19EF19BC19FF19CC1A0F12B
:100920009DC1A1F19EC1A2F19FC1A3F1A0C1A4F1FB
:10093000A1C1A5F1A2C1A6F1A3C1A7F1A4C1A8F1CB
:10094000A5C1A9F1A6C1AAF1A7C1ABF1A8C1ACF19B
:10095000A9C1ADF1AAC1AEF1ABC1AFF1ACC1B0F16B
:10096000ADC1B1F1AEC1B2F1AFC1B3F1B0C1B4F13B
:10097000B1C1B5F101015E6B5F6B606B616B96514C
:100980005E2797515F2398516023995161239A51B3
:100990005E279B515F239C5160239D5161239E5193
:1009A0005E279F515F23A0516023A1516123A25173
:1009B0005E27A3515F23A4516023A5516123A65153
:1009C0005E27A7515F23A8516023A9516123AA5133
:1009D0005E27AB515F23AC516023AD516123AE5113
:1009E0005E27AF515F23B0516023B1516123B251F3
:1009F0005E27B3515F23B4516023B5516123D89072
:100A0000613360335F335E33D890613360335F337B
:100A10005E33D890613360335F335E3393EF07F01A
:100A20000392030103EE00F080517F0BE92604C01E
:100A3000EFFF802B8151805D700BD8A48B8200006A
:100A40008051815D700BD8A48B9281518019D8B4EC
:100A5000079093EF07F0F2940101453F93EF07F001
:100A6000462B93EF07F09E900101533F93EF07F061
:100A7000542B93EF07F09E9204005CA140EF05F029
:100A8000077C07AC5BEF05F0C274C2B455EF05F00C
:100A9000C3CFADF5C4CFAEF50501D890AE33AD33BD
:100AA000D890AE33AD335CEF05F0C3CF55F1C4CF72
:100AB00056F15CEF05F0C28207B4C9EF05F047C1FB
:100AC0004BF148C14CF149C14DF14AC14EF15EC1F3
:100AD00062F15FC163F160C164F161C165F196C10A
:100AE000B6F197C1B7F198C1B8F199C1B9F19AC1FE
:100AF000BAF19BC1BBF19CC1BCF19DC1BDF19EC1CE
:100B0000BEF19FC1BFF1A0C1C0F1A1C1C1F1A2C19D
:100B1000C2F1A3C1C3F1A4C1C4F1A5C1C5F1A6C16D
:100B2000C6F1A7C1C7F1A8C1C8F1A9C1C9F1AAC13D
:100B3000CAF1ABC1CBF1ACC1CCF1ADC1CDF1AEC10D
:100B4000CEF1AFC1CFF1B0C1D0F1B1C1D1F1B2C1DD
:100B5000D2F1B3C1D3F1B4C1D4F1B5C1D5F1ADC5B2
:100B6000AFF5AEC5B0F5AFC5B1F5B0C5B2F5010191
:100B700055515B2756515C23E86A5D230E2EC9EF61
:100B800005F05CC157F15DC158F15B6B5C6B5D6B4F
:100B9000078E0201002F93EF07F03C0E006F00C19B
:100BA0000CF101C10DF102C10EF103C10FF104C13D
:100BB00010F105C111F106C112F107C113F108C10D
:100BC00014F109C115F10AC116F10BC117F134C1B5
:100BD00035F105012951000AD8B492EF06F005015C
:100BE0002951010AD8B41CEF06F005012951020A67
:100BF000D8B45DEF06F005012951030AD8B45DEFC2
:100C000006F005012951040AD8B45DEF06F005018C
:100C10002951050AD8B45DEF06F005012951060AED
:100C2000D8B45DEF06F005012951070AD8B45DEF8D
:100C300006F0296B92EF06F005014D6727EF06F0ED
:100C40004E6727EF06F04F6727EF06F050672BEF50
:100C500006F092EF06F051C500F152C501F153C5FF
:100C600002F154C503F10101010E046F000E056F7E
:100C7000000E066F000E076F7DEC20F000C151F5ED
:100C800001C152F502C153F503C154F5006750EF9D
:100C900006F0016750EF06F0026750EF06F00367B9
:100CA00092EF06F04DC551F54EC552F54FC553F5BF
:100CB00050C554F50F8892EF06F005012A6763EFDF
:100CC00006F092EF06F00FBE78EF06F010A07DEF71
:100CD00006F00101476774EF06F0486774EF06F00D
:100CE000496774EF06F04A6778EF06F07DEF06F08B
:100CF00007AE7DEF06F08FEF06F005012B2F92EF88
:100D000006F03C0E2B6F2A2F92EF06F00101000E29
:100D1000626FE00E636FA50E646F010E656F0501D3
:100D20002A6B0F8805015C6B2DB798EF06F05C818C
:100D30000CC100F10DC101F10EC102F10FC103F1AF
:100D400010C104F111C105F112C106F113C107F17F
:100D500014C108F115C109F116C10AF117C10BF14F
:100D600035C134F100C10CF101C10DF102C10EF128
:100D700003C10FF104C110F105C111F106C112F157
:100D800007C113F108C114F109C115F10AC116F127
:100D90000BC117F134C135F101018A67D7EF06F0B5
:100DA0008B67D7EF06F08C67D7EF06F08D67DBEF28
:100DB00006F00BEF07F08EC100F18FC101F190C179
:100DC00002F191C103F10101010E046F000E056FE4
:100DD000000E066F000E076F7DEC20F000C18EF153
:100DE00001C18FF102C190F103C191F1006700EFE1
:100DF00007F0016700EF07F0026700EF07F00367F5
:100E00000BEF07F08AC18EF18BC18FF18CC190F18D
:100E10008DC191F10F80D57ED5BE69D0D6CF47F177
:100E2000D7CF48F145C149F1E86AE8CF4AF11090BF
:100E300047C100F148C101F149C102F14AC103F1C2
:100E400001010A0E046F000E056F000E066F000E02
:100E5000076F7DEC20F000AF1080010154A73DEF3B
:100E600007F00F9A0F9C0F9E0101000E5E6F600E3F
:100E70005F6F3D0E606F080E616F010147BF4DEF60
:100E800007F048674DEF07F049674DEF07F04A67F5
:100E90004DEF07F0F28872EF07F0F2985E6B5F6B30
:100EA000606B616B966B976B986B996B9A6B9B6B96
:100EB0009C6B9D6B9E6B9F6BA06BA16BA26BA36BDE
:100EC000A46BA56BA66BA76BA86BA96BAA6BAB6B8E
:100ED000AC6BAD6BAE6BAF6BB06BB16BB26BB36B3E
:100EE000B46BB56BD76AD66A0101456B466B0CC112
:100EF00000F10DC101F10EC102F10FC103F110C1EA
:100F000004F111C105F112C106F113C107F114C1B9
:100F100008F115C109F116C10AF117C10BF135C16C
:100F200034F193EF07F002C0E0FF005001C0D8FF9A
:100F30001000A6B299EF07F00CC0A9FF0BC0A8FFE4
:100F4000A69EA69CA684F29E550EA76EAA0EA76E1C
:100F5000A682F28EA694A6B2ABEF07F00C2A12007E
:100F6000A96EA69EA69CA680A8500C2A1200040179
:100F70002C0E826FA4EC0AF074EC21F00C50B0EC53
:100F800007F0E8CF00F10C50B0EC07F0E8CF01F12A
:100F900001AFD0EF07F00101FF0E026FFF0E036FEC
:100FA00017EC21F02967DCEF07F00401200E826FB7
:100FB000A4EC0AF0E1EF07F004012D0E826FA4EC1F
:100FC0000AF045EC1FF01200076A0F6A106A0F0161
:100FD0000D0EC16E860EC06E030EC26E0F01280E7E
:100FE000896E130E926E080E8A6EF30E936E0C0EBF
:100FF0008A6EF10E936E8B6A900E946EF18EF19E56
:101000000E6A01015B6B5C6B5D6B576B586BF29A00
:101010000101476B486B496B4A6B4B6B4C6B4D6BDB
:101020004E6B4F6B506B516B526B456B466BD76A77
:10103000D66A0F01280ED56EF28A9D90B00ECD6E45
:1010400001015E6B5F6B606B616B626B636B646B0A
:10105000656B666B676B686B696B536B546BCF6AC0
:10106000CE6A0F9A0F9C0F9E9D80760ECA6E9D824F
:1010700002013C0E006FCC6A160EB0EC07F0E8CF10
:1010800000F1170EB0EC07F0E8CF01F1180EB0EC4C
:1010900007F0E8CF02F1190EB0EC07F0E8CF03F14A
:1010A000010103AF6EEF08F074EC21F0160E0C6E28
:1010B00000C10BF099EC07F0170E0C6E01C10BF09C
:1010C00099EC07F0180E0C6E02C10BF099EC07F0CA
:1010D000190E0C6E03C10BF099EC07F000C18AF1F8
:1010E00001C18BF102C18CF103C18DF100C18EF100
:1010F00001C18FF102C190F103C191F11A0EB0EC60
:1011000007F0E8CF00F11B0EB0EC07F0E8CF01F1DB
:101110001C0EB0EC07F0E8CF02F11D0EB0EC07F0AA
:10112000E8CF03F1010103AFC4EF08F074EC21F044
:101130001A0E0C6E00C10BF099EC07F01B0E0C6E32
:1011400001C10BF099EC07F01C0E0C6E02C10BF004
:1011500099EC07F01D0E0C6E03C10BF099EC07F033
:101160001A0EB0EC07F0E8CF00F11B0EB0EC07F060
:10117000E8CF01F11C0EB0EC07F0E8CF02F11D0E34
:10118000B0EC07F0E8CF03F100C192F101C193F197
:1011900002C194F103C195F1240EAC6E900EAB6EBA
:1011A000240EAC6E080EB86E000EB06E1F0EAF6E41
:1011B0000401806B816B0F01900EAB6E0F019D8A55
:1011C0000301806B816BC26B8B92E4EC25F0200EE7
:1011D000B0EC07F0E8CF29F505012951FF0AD8A4A2
:1011E000F9EF08F0296B200E0C6E29C50BF099EC75
:1011F00007F00501010E2A6F3C0E2B6F250EB0EC97
:1012000007F0E8CF00F1260EB0EC07F0E8CF01F1CF
:10121000270EB0EC07F0E8CF02F1280EB0EC07F093
:10122000E8CF03F1010103AF30EF09F074EC21F0D6
:10123000250E0C6E00C10BF099EC07F0260E0C6E1B
:1012400001C10BF099EC07F0270E0C6E02C10BF0F8
:1012500099EC07F0280E0C6E03C10BF099EC07F027
:1012600000C14DF501C14EF502C14FF503C150F566
:1012700000C151F501C152F502C153F503C154F546
:10128000290EB0EC07F0E8CF55F505015651555D34
:10129000D8A055C556F505012951020A0EE181B8BD
:1012A0005DEF09F00501562F5AEF09F055C556F5C7
:1012B0005DEF09F081BAB2EF27F0210EB0EC07F034
:1012C000E8CF00F1220EB0EC07F0E8CF01F1230ED9
:1012D000B0EC07F0E8CF02F1240EB0EC07F0E8CF55
:1012E00003F1010103AFA3EF09F074EC21F0210E2B
:1012F0000C6E00C10BF099EC07F0220E0C6E01C1D0
:101300000BF099EC07F0230E0C6E02C10BF099EC78
:1013100007F0240E0C6E03C10BF099EC07F0210EC0
:10132000B0EC07F0E8CF00F1220EB0EC07F0E8CF08
:1013300001F1230EB0EC07F0E8CF02F1240EB0EC7F
:1013400007F0E8CF03F100C157F501C158F502C11C
:1013500059F503C15AF51BEC25F0DDEC23F02DEC1B
:1013600023F005012951030A12E005012951040A5D
:101370001DE005012951050A24E005012951060A4D
:1013800032E005012951070A38E006EF0AF0A6C548
:1013900000F101010F0E001701010051000A36E0B3
:1013A00001010051050A32E003EF0AF0A6C500F181
:1013B00001010F0E001701010051000A27E003EFA1
:1013C0000AF00501A651000A21E00501A651150AFF
:1013D0001DE00501A651300A19E00501A651450A94
:1013E00015E003EF0AF00501A651000A0FE0050120
:1013F000A651300A0BE003EF0AF00501A651000ADE
:1014000005E003EF0AF081BAB2EF27F08A86D8EC44
:1014100022F007900001F28EF28C07B0D0EF1DF0A1
:101420000FB0B1EF18F00FB8A3EF12F00301805125
:1014300081197F0BD8B4D0EF1DF013EE00F081516D
:101440007F0BE126812BE7CFE8FFE00BD8B4D0EF8C
:101450001DF023EE82F0C2513F0BD926E7CFDFFF0C
:10146000C22BDF50780AD8A4D0EF1DF007808EC1C0
:1014700000F18FC101F190C102F191C103F10101AD
:10148000040E046F000E056F000E066F000E076F4E
:101490007DEC20F000AF56EF0AF00101030E8E6FD5
:1014A000000E8F6F000E906F000E916F030182513E
:1014B000720AD8B4B1EF18F08251520AD8B4B1EF21
:1014C00018F08251750AD8B4B1EF18F08251630A4E
:1014D000D8B48CEF1AF08251690AD8B46CEF15F0C9
:1014E00082517A0AD8B47FEF16F08251490AD8B4F3
:1014F0000BEF15F08251500AD8B429EF14F0825145
:10150000700AD8B46CEF14F08251540AD8B497EF33
:1015100014F08251740AD8B4DDEF14F08251730ACA
:10152000D8B4E1EF17F08251530AD8B446EF18F05F
:1015300082514C0AD8B449EF0EF08251760AD8B4E1
:10154000B7EF0AF0C1EF1AF0040114EE00F0805179
:101550007F0BE12682C4E7FF802B12000D0E826F05
:10156000A4EC0AF00A0E826FA4EC0AF01200030148
:101570008351300AD8B4D8EF0AF003018351310AFD
:10158000D8B40FEF0BF003018351320AD8B4E5EF62
:101590000BF003018351330AD8B4BBEF0CF0030105
:1015A0008351340AD8B461EF0DF0D8A4C1EF1AF01A
:1015B0000401760E826FA4EC0AF00401300E826FF3
:1015C000A4EC0AF004012C0E826FA4EC0AF0E2EC09
:1015D00021F074EC21F000C600F101C601F117EC16
:1015E00021F030C182F40401300E8227A4EC0AF00D
:1015F00031C182F40401300E8227A4EC0AF032C11A
:1016000082F40401300E8227A4EC0AF033C182F484
:101610000401300E8227A4EC0AF0D6EF12F0040188
:10162000760E826FA4EC0AF00401310E826FA4ECF6
:101630000AF004012C0E826FA4EC0AF008EC22F0F0
:1016400008EC22F074EC21F002C600F103C601F1AF
:1016500001AF30EF0BF00101FF0E026FFF0E036FC1
:1016600017EC21F0296737EF0BF03CEF0BF004018A
:101670002D0E826FA4EC0AF02FC182F40401300E0B
:101680008227A4EC0AF030C182F40401300E8227D4
:10169000A4EC0AF031C182F40401300E8227A4ECDC
:1016A0000AF032C182F40401300E8227A4EC0AF061
:1016B00033C182F40401300E8227A4EC0AF0040145
:1016C0002C0E826FA4EC0AF074EC21F004C600F139
:1016D00005C601F101AF72EF0BF00101FF0E026FC1
:1016E000FF0E036F17EC21F0296779EF0BF07EEF07
:1016F0000BF004012D0E826FA4EC0AF02FC182F4CE
:101700000401300E8227A4EC0AF030C182F40401F7
:10171000300E8227A4EC0AF031C182F40401300EAD
:101720008227A4EC0AF032C182F40401300E822731
:10173000A4EC0AF033C182F40401300E8227A4EC39
:101740000AF004012C0E826FA4EC0AF074EC21F074
:1017500006C600F107C601F101AFB4EF0BF00101BD
:10176000FF0E026FFF0E036F17EC21F02967BBEF2E
:101770000BF0C0EF0BF004012D0E826FA4EC0AF009
:101780002FC182F40401300E8227A4EC0AF030C18C
:1017900082F40401300E8227A4EC0AF031C182F4F5
:1017A0000401300E8227A4EC0AF032C182F4040155
:1017B000300E8227A4EC0AF033C182F40401300E0B
:1017C0008227A4EC0AF0D6EF12F00401760E826FA5
:1017D000A4EC0AF00401320E826FA4EC0AF00401BA
:1017E0002C0E826FA4EC0AF070EC22F070EC22F068
:1017F00074EC21F008C600F109C601F101AF06EF53
:101800000CF00101FF0E026FFF0E036F17EC21F0C9
:1018100029670DEF0CF012EF0CF004012D0E826F12
:10182000A4EC0AF02FC182F40401300E8227A4EC4C
:101830000AF030C182F40401300E8227A4EC0AF0D1
:1018400031C182F40401300E8227A4EC0AF032C1C7
:1018500082F40401300E8227A4EC0AF033C182F432
:101860000401300E8227A4EC0AF004012C0E826FD2
:10187000A4EC0AF074EC21F00AC600F10BC601F1E9
:1018800001AF48EF0CF00101FF0E026FFF0E036F76
:1018900017EC21F029674FEF0CF054EF0CF0040126
:1018A0002D0E826FA4EC0AF02FC182F40401300ED9
:1018B0008227A4EC0AF030C182F40401300E8227A2
:1018C000A4EC0AF031C182F40401300E8227A4ECAA
:1018D0000AF032C182F40401300E8227A4EC0AF02F
:1018E00033C182F40401300E8227A4EC0AF0040113
:1018F0002C0E826FA4EC0AF074EC21F00CC600F1FF
:101900000DC601F101AF8AEF0CF00101FF0E026F6D
:10191000FF0E036F17EC21F0296791EF0CF096EFA3
:101920000CF004012D0E826FA4EC0AF02FC182F49A
:101930000401300E8227A4EC0AF030C182F40401C5
:10194000300E8227A4EC0AF031C182F40401300E7B
:101950008227A4EC0AF032C182F40401300E8227FF
:10196000A4EC0AF033C182F40401300E8227A4EC07
:101970000AF0D6EF12F00401760E826FA4EC0AF0A2
:101980000401330E826FA4EC0AF004012C0E826F66
:10199000A4EC0AF085C382F4A4EC0AF0640E0D6E88
:1019A00003018551320A02E16A0E0D6E0301855171
:1019B000330A02E1700E0D6E03018551340A02E113
:1019C000760E0D6E03018551350A02E17C0E0D6E17
:1019D00003018551360A02E1820E0D6E0301865124
:1019E000780A65E00DC00CF0B5EC21F02981030107
:1019F00087512D0AD8B4FFEF0CF00101299188C35B
:101A00002FF189C330F18AC331F18BC332F18CC31A
:101A100033F1C2EC21F039EC21F000C10BF099EC6C
:101A200007F001C10BF099EC07F0B5EC21F029812A
:101A300003018E512D0AD8B420EF0DF00101299138
:101A40008FC32FF190C330F191C331F192C332F1C2
:101A500093C333F1C2EC21F039EC21F000C10BF05B
:101A600099EC07F001C10BF099EC07F0B5EC21F00F
:101A70002981030195512D0AD8B441EF0DF00101E0
:101A8000299196C32FF197C330F198C331F199C3CF
:101A900032F19AC333F1C2EC21F039EC21F000C1EC
:101AA0000BF099EC07F001C10BF099EC07F00DC0B9
:101AB0000CF0B7EC07F0B7EC07F0B7EC07F0D6EF97
:101AC00012F00401760E826FA4EC0AF00401340EC9
:101AD000826FA4EC0AF003018451780AD8B439EF7C
:101AE0000EF03E0E0C6EB5EC21F0298103018551FC
:101AF0002D0AD8B47EEF0DF00101299186C32FF194
:101B000087C330F188C331F189C332F18AC333F11D
:101B1000C2EC21F039EC21F000C10BF099EC07F098
:101B200001C10BF099EC07F0B5EC21F0298103011C
:101B30008C512D0AD8B49FEF0DF0010129918DC36E
:101B40002FF18EC330F18FC331F190C332F191C3C5
:101B500033F1C2EC21F039EC21F000C10BF099EC2B
:101B600007F001C10BF099EC07F0B5EC21F02981E9
:101B7000030193512D0AD8B4C0EF0DF00101299152
:101B800094C32FF195C330F196C331F197C332F16D
:101B900098C333F1C2EC21F039EC21F000C10BF015
:101BA00099EC07F001C10BF099EC07F0B5EC21F0CE
:101BB000298103019A512D0AD8B4E1EF0DF00101FA
:101BC00029919BC32FF19CC330F19DC331F19EC37A
:101BD00032F19FC333F1C2EC21F039EC21F000C1A6
:101BE0000BF099EC07F001C10BF099EC07F0B5ECA4
:101BF00021F029810301A1512D0AD8B402EF0EF082
:101C000001012991A2C32FF1A3C330F1A4C331F183
:101C1000A5C332F1A6C333F1C2EC21F039EC21F0B7
:101C200000C10BF099EC07F001C10BF099EC07F043
:101C3000B5EC21F029810301A8512D0AD8B423EF76
:101C40000EF001012991A9C32FF1AAC330F1ABC352
:101C500031F1ACC332F1ADC333F1C2EC21F039EC58
:101C600021F000C10BF099EC07F001C10BF099ECE9
:101C700007F03E0E0C6EB7EC07F0B7EC07F0B7ECD0
:101C800007F0B7EC07F0B7EC07F0B7EC07F0D6EFCA
:101C900012F003018351300AD8B4F8EF10F00301B9
:101CA0008351310AD8B47EEF11F003018351320A17
:101CB000D8B4CEEF11F003018351330AD8B4D2EF78
:101CC00011F003018351340AD8B4E0EF11F003019D
:101CD0008351350AD8B4A8EF12F0030183514D0A9D
:101CE000D8B471EF0FF0030183516D0AD8B48BEFB4
:101CF0000FF003018351490AD8B4A8EF13F0030190
:101D00008351500AD8B4DAEF12F003018351540A18
:101D1000D8B453EF13F003018351630AD8B4ABEF87
:101D20000FF003018351430AD8B4A3EF10F003016D
:101D30008351730AD8B4A9EF0FF003018351610AEC
:101D4000D8B4BEEF0EF003018351650AD8B446EF54
:101D500011F003018351450AD8B454EF11F0030187
:101D60008351620AD8B462EF11F003018351420A31
:101D7000D8B470EF11F0D8A4C1EF1AF004014C0EE2
:101D8000826FA4EC0AF00401610E826FA4EC0AF0E9
:101D9000DDEC23F004012C0E826FA4EC0AF074EC4D
:101DA00021F0A5C500F1010117EC21F031C182F449
:101DB0000401300E8227A4EC0AF032C182F404013F
:101DC000300E8227A4EC0AF033C182F40401300EF5
:101DD0008227A4EC0AF004012C0E826FA4EC0AF016
:101DE00074EC21F0A6C500F1010117EC21F031C11E
:101DF00082F40401300E8227A4EC0AF032C182F48E
:101E00000401300E8227A4EC0AF033C182F40401ED
:101E1000300E8227A4EC0AF004012C0E826FA4EC91
:101E20000AF074EC21F0A7C500F1010117EC21F0D4
:101E300031C182F40401300E8227A4EC0AF032C1D1
:101E400082F40401300E8227A4EC0AF033C182F43C
:101E50000401300E8227A4EC0AF004012C0E826FDC
:101E6000A4EC0AF074EC21F0A8C500F1010117EC14
:101E700021F031C182F40401300E8227A4EC0AF073
:101E800032C182F40401300E8227A4EC0AF033C17F
:101E900082F40401300E8227A4EC0AF004012C0E17
:101EA000826FA4EC0AF074EC21F0ADC500F10101E1
:101EB00017EC21F031C182F40401300E8227A4EC2A
:101EC0000AF032C182F40401300E8227A4EC0AF039
:101ED00033C182F40401300E8227A4EC0AF0D6EF5D
:101EE00012F0B5EC21F084C333F1C2EC21F039ECEF
:101EF00021F0200E0C6E00C10BF099EC07F000C130
:101F000029F505012951000A06E005012951010AB8
:101F100002E083EC24F004014C0E826FA4EC0AF082
:101F200004014D0E826FA4EC0AF004012C0E826FA6
:101F3000A4EC0AF074EC21F029C500F117EC21F0B3
:101F400033C182F40401300E8227A4EC0AF0D6EFEC
:101F500012F0B2EF27F004014C0E826FA4EC0AF0ED
:101F60000401630E826FA4EC0AF02DEC23F004014F
:101F70002C0E826FA4EC0AF0C0EC0FF0D6EF12F03A
:101F800074EC21F0ABC500F10101003B0F0E00170E
:101F900017EC21F033C182F40401300E8227A4EC47
:101FA0000AF0ABC500F101010F0E0101001717EC9B
:101FB00021F033C182F40401300E8227A4EC0AF030
:101FC00004012D0E826FA4EC0AF0AAC500F10101F4
:101FD000003B0F0E001717EC21F033C182F404010F
:101FE000300E8227A4EC0AF0AAC500F101010F0E01
:101FF0000101001717EC21F033C182F40401300E07
:102000008227A4EC0AF004012D0E826FA4EC0AF0E2
:10201000A9C500F10101003B0F0E001717EC21F0DC
:1020200033C182F40401300E8227A4EC0AF0A9C562
:1020300000F101010F0E0101001717EC21F033C16F
:1020400082F40401300E8227A4EC0AF00401200E71
:10205000826FA4EC0AF0A8C500F10F0E0101001771
:1020600017EC21F033C182F40401300E8227A4EC76
:102070000AF00401200E826FA4EC0AF0A7C500F15B
:1020800001010101003B0F0E001717EC21F033C1D5
:1020900082F40401300E8227A4EC0AF0A7C500F1F7
:1020A00001010F0E0101001717EC21F033C182F47A
:1020B0000401300E8227A4EC0AF004013A0E826F6C
:1020C000A4EC0AF0A6C500F10101003B0F0E0017B9
:1020D00017EC21F033C182F40401300E8227A4EC06
:1020E0000AF0A6C500F101010F0E0101001717EC5F
:1020F00021F033C182F40401300E8227A4EC0AF0EF
:1021000004013A0E826FA4EC0AF0A5C500F10101AA
:10211000003B0F0E001717EC21F033C182F40401CD
:10212000300E8227A4EC0AF0A5C500F101010F0EC4
:10213000001717EC21F033C182F40401300E82271E
:10214000A4EC0AF0120084C3E8FF0F0BE83AE8CFD2
:10215000ABF585C3E8FF0F0B0501AB1387C3E8FFA1
:102160000F0BE83AE8CFAAF588C3E8FF0F0B05018B
:10217000AA138AC3E8FF0F0BE83AE8CFA9F58BC38F
:10218000E8FF0F0B0501A9138DC3E8FF0F0BE8CF84
:10219000A8F58FC3E8FF0F0BE83AE8CFA7F590C387
:1021A000E8FF0F0B0501A71392C3E8FF0F0BE83AF6
:1021B000E8CFA6F593C3E8FF0F0B0501A61395C35F
:1021C000E8FF0F0BE83AE8CFA5F596C3E8FF0F0B41
:1021D0000501A5138CEC23F004014C0E826FA4ECD6
:1021E0000AF00401430E826FA4EC0AF0B5EF0FF081
:1021F00073EC27F074EC21F02DC500F117EC21F001
:1022000004014C0E826FA4EC0AF00401300E826FC0
:10221000A4EC0AF004012C0E826FA4EC0AF031C188
:1022200082F40401300E8227A4EC0AF032C182F459
:102230000401300E8227A4EC0AF033C182F40401B9
:10224000300E8227A4EC0AF004012C0E826FA4EC5D
:102250000AF074EC21F02EC500F117EC21F031C129
:1022600082F40401300E8227A4EC0AF032C182F419
:102270000401300E8227A4EC0AF033C182F4040179
:10228000300E8227A4EC0AF0D6EF12F004014C0EB7
:10229000826FA4EC0AF00401650E826FA4EC0AF0D0
:1022A0006CEC25F0D6EF12F004014C0E826FA4EC1A
:1022B0000AF00401450E826FA4EC0AF089EC25F0C7
:1022C000D6EF12F004014C0E826FA4EC0AF0040168
:1022D000620E826FA4EC0AF0C3EC25F0D6EF12F088
:1022E00004014C0E826FA4EC0AF00401420E826FCE
:1022F000A4EC0AF0A6EC25F0D6EF12F004014C0E87
:10230000826FA4EC0AF00401310E826FA4EC0AF093
:1023100004012C0E826FA4EC0AF025C500F126C53D
:1023200001F127C502F128C503F10101100E046F68
:10233000000E056F000E066F000E076FABEC20F06D
:1023400017EC21F02EC182F40401300E8227A4EC98
:102350000AF02FC182F40401300E8227A4EC0AF0A7
:1023600030C182F40401300E8227A4EC0AF031C19E
:1023700082F40401300E8227A4EC0AF032C182F408
:102380000401300E8227A4EC0AF033C182F4040168
:10239000300E8227A4EC0AF0D6EF12F02EEC26F0D5
:1023A000C1EF1AF004014C0E826FA4EC0AF0040194
:1023B000330E826FA4EC0AF064EC26F088EF11F083
:1023C00004014C0E826FA4EC0AF00401340E826FFB
:1023D000A4EC0AF004012C0E826FA4EC0AF0B5EC18
:1023E00021F084C32AF185C32BF186C32CF187C366
:1023F0002DF188C32EF189C32FF18AC330F18BC32D
:1024000031F18CC332F18DC333F10101296BC2EC80
:1024100021F039EC21F0100E046F000E056F000E54
:10242000066F000E076F8CEC20F000C121F501C192
:1024300022F502C123F503C124F526EC27F02EC5B1
:10244000A5F52FC5A6F530C5A7F531C5A8F532C548
:10245000A9F533C5AAF534C5ABF5C0EC0FF00401FE
:102460002C0E826FA4EC0AF035C500F136C501F1DF
:1024700037C502F138C503F10101000E046F000EEB
:10248000056F010E066F000E076FABEC20F017EC26
:1024900021F029674EEF12F053EF12F004012D0ED8
:1024A000826FA4EC0AF030C182F40401300E82275E
:1024B000A4EC0AF031C182F40401300E8227A4ECAE
:1024C0000AF004012E0E826FA4EC0AF032C182F4ED
:1024D0000401300E8227A4EC0AF033C182F4040117
:1024E000300E8227A4EC0AF004012C0E826FA4ECBB
:1024F0000AF074EC21F039C500F13AC501F1EBECBA
:102500001BF004012C0E826FA4EC0AF074EC21F095
:102510003BC500F117EC21F031C182F40401300E0B
:102520008227A4EC0AF032C182F40401300E822723
:10253000A4EC0AF033C182F40401300E8227A4EC2B
:102540000AF0D6EF12F00F9864EC26F0D6EF12F0F6
:1025500004014C0E826FA4EC0AF00401350E826F68
:10256000A4EC0AF004012C0E826FA4EC0AF074ECC7
:1025700021F00784AFC500F1079417EC21F031C1B9
:1025800082F40401300E8227A4EC0AF032C182F4F6
:102590000401300E8227A4EC0AF033C182F4040156
:1025A000300E8227A4EC0AF0D6EF12F0AEEC0AF05F
:1025B000C1EF1AF004014C0E826FA4EC0AF0040182
:1025C000500E826FA4EC0AF004012C0E826FA4EC72
:1025D0000AF085C32AF186C32BF187C32CF188C387
:1025E0002DF189C32EF18AC32FF18BC330F18CC337
:1025F00031F18DC332F18EC333F10101C2EC21F010
:1026000039EC21F003018451530A0DE00301845198
:102610004D0A38E00401780E826FA4EC0AF0AEECAB
:102620000AF0C1EF1AF00401530E826FA4EC0AF015
:10263000250E0C6E00C10BF099EC07F0260E0C6E07
:1026400001C10BF099EC07F0270E0C6E02C10BF0E4
:1026500099EC07F0280E0C6E03C10BF099EC07F013
:1026600000C14DF501C14EF502C14FF503C150F552
:1026700000C151F501C152F502C153F503C154F532
:10268000B7EF13F004014D0E826FA4EC0AF0290E8F
:102690000C6E00C10BF099EC07F000C155F500C1BC
:1026A00056F5B7EF13F004014C0E826FA4EC0AF05C
:1026B0000401540E826FA4EC0AF004012C0E826F08
:1026C000A4EC0AF084C32AF185C32BF186C32CF154
:1026D00087C32DF188C32EF189C32FF18AC330F14E
:1026E0008BC331F18DC332F18EC333F10101C2ECE2
:1026F00021F039EC21F00101000E046F000E056F8E
:10270000010E066F000E076F8CEC20F0210E0C6E90
:1027100000C10BF099EC07F0220E0C6E01C10BF01A
:1027200099EC07F0230E0C6E02C10BF099EC07F048
:10273000240E0C6E03C10BF099EC07F000C157F5A5
:1027400001C158F502C159F503C15AF5B7EF13F0AD
:1027500004014C0E826FA4EC0AF00401490E826F52
:10276000A4EC0AF004012C0E826FA4EC0AF0250EF2
:10277000B0EC07F0E8CF00F1260EB0EC07F0E8CFA0
:1027800001F1270EB0EC07F0E8CF02F1280EB0EC13
:1027900007F0E8CF03F117EC21F0FEEC1EF0040186
:1027A000730E826FA4EC0AF004012C0E826FA4EC6D
:1027B0000AF074EC21F0290EB0EC07F0E8CF00F13C
:1027C00017EC21F0FEEC1EF00401730E826FA4ECF6
:1027D0000AF004012C0E826FA4EC0AF051C500F13E
:1027E00052C501F153C502F154C503F117EC21F0B4
:1027F000FEEC1EF00401730E826FA4EC0AF00401DB
:102800002C0E826FA4EC0AF074EC21F056C500F196
:1028100017EC21F0FEEC1EF004016D0E826FA4ECAB
:102820000AF004012C0E826FA4EC0AF057C500F1E7
:1028300058C501F159C502F15AC503F1DCEC1AF093
:1028400004012C0E826FA4EC0AF0AEEC0AF0C1EF8A
:102850001AF083C32AF184C32BF185C32CF186C3FC
:102860002DF187C32EF188C32FF189C330F18AC3BC
:1028700031F18BC332F18CC333F10101C2EC21F091
:1028800039EC21F0160E0C6E00C10BF099EC07F03C
:10289000170E0C6E01C10BF099EC07F0180E0C6EC0
:1028A00002C10BF099EC07F0190E0C6E03C10BF08E
:1028B00099EC07F000C18AF101C18BF102C18CF1E2
:1028C00003C18DF100C18EF101C18FF102C190F100
:1028D00003C191F10BEF15F083C32AF184C32BF1EF
:1028E00085C32CF186C32DF187C32EF188C32FF148
:1028F00089C330F18AC331F18BC332F18CC333F118
:102900000101C2EC21F039EC21F000C18AF101C1D2
:102910008BF102C18CF103C18DF100C18EF101C1B7
:102920008FF102C190F103C191F10BEF15F083C358
:102930002AF184C32BF185C32CF186C32DF187C303
:102940002EF188C32FF189C330F18AC331F18CC3D2
:1029500032F18DC333F10101C2EC21F039EC21F0E9
:102960000101000E046F000E056F010E066F000ED0
:10297000076F8CEC20F01A0E0C6E00C10BF099EC76
:1029800007F01B0E0C6E01C10BF099EC07F01C0E4A
:102990000C6E02C10BF099EC07F01D0E0C6E03C11A
:1029A0000BF099EC07F000C192F101C193F102C163
:1029B00094F103C195F10BEF15F083C32AF184C3A1
:1029C0002BF185C32CF186C32DF187C32EF188C36B
:1029D0002FF189C330F18AC331F18CC332F18DC339
:1029E00033F10101C2EC21F039EC21F00101000EBC
:1029F000046F000E056F010E066F000E076F8CEC62
:102A000020F000C192F101C193F102C194F103C120
:102A100095F10BEF15F0160EB0EC07F0E8CF00F1D2
:102A2000170EB0EC07F0E8CF01F1180EB0EC07F08C
:102A3000E8CF02F1190EB0EC07F0E8CF03F117EC84
:102A400021F0FEEC1EF00401730E826FA4EC0AF07C
:102A500004012C0E826FA4EC0AF08AC100F18BC134
:102A600001F18CC102F18DC103F117EC21F0FEECF4
:102A70001EF00401730E826FA4EC0AF004012C0E08
:102A8000826FA4EC0AF01A0EB0EC07F0E8CF00F168
:102A90001B0EB0EC07F0E8CF01F11C0EB0EC07F014
:102AA000E8CF02F11D0EB0EC07F0E8CF03F1DCEC4B
:102AB0001AF004012C0E826FA4EC0AF092C100F10E
:102AC00093C101F194C102F195C103F1DCEC1AF05C
:102AD000AEEC0AF0C1EF1AF00401690E826FA4ECAB
:102AE0000AF004012C0E826FA4EC0AF00101040E1E
:102AF000006F000E016F000E026F000E036F17ECE7
:102B000021F02CC182F40401300E8227A4EC0AF0DB
:102B10002DC182F40401300E8227A4EC0AF02EC1EC
:102B200082F40401300E8227A4EC0AF02FC182F453
:102B30000401300E8227A4EC0AF030C182F40401B3
:102B4000300E8227A4EC0AF031C182F40401300E69
:102B50008227A4EC0AF032C182F40401300E8227ED
:102B6000A4EC0AF033C182F40401300E8227A4ECF5
:102B70000AF004012C0E826FA4EC0AF001010B0E86
:102B8000006F000E016F000E026F000E036F17EC56
:102B900021F02CC182F40401300E8227A4EC0AF04B
:102BA0002DC182F40401300E8227A4EC0AF02EC15C
:102BB00082F40401300E8227A4EC0AF02FC182F4C3
:102BC0000401300E8227A4EC0AF030C182F4040123
:102BD000300E8227A4EC0AF031C182F40401300ED9
:102BE0008227A4EC0AF032C182F40401300E82275D
:102BF000A4EC0AF033C182F40401300E8227A4EC65
:102C00000AF004012C0E826FA4EC0AF001011A0EE6
:102C1000006F000E016F000E026F000E036F17ECC5
:102C200021F02CC182F40401300E8227A4EC0AF0BA
:102C30002DC182F40401300E8227A4EC0AF02EC1CB
:102C400082F40401300E8227A4EC0AF02FC182F432
:102C50000401300E8227A4EC0AF030C182F4040192
:102C6000300E8227A4EC0AF031C182F40401300E48
:102C70008227A4EC0AF032C182F40401300E8227CC
:102C8000A4EC0AF033C182F40401300E8227A4ECD4
:102C90000AF004012C0E826FA4EC0AF0200EF86EEC
:102CA000F76AF66A04010900F5CF82F4A4EC0AF091
:102CB0000900F5CF82F4A4EC0AF00900F5CF82F404
:102CC000A4EC0AF00900F5CF82F4A4EC0AF00900A4
:102CD000F5CF82F4A4EC0AF00900F5CF82F4A4EC5D
:102CE0000AF00900F5CF82F4A4EC0AF00900F5CF50
:102CF00082F4A4EC0AF0AEEC0AF0C1EF1AF08351B2
:102D0000630AD8A4C1EF1AF08451610AD8A4C1EFB4
:102D10001AF085516C0AD8A4C1EF1AF08651410A05
:102D200042E08651440A1BE08651420AD8B4E6EFDD
:102D300016F08651350AD8B44BEF1CF08651360A8E
:102D4000D8B4A0EF1CF08651370AD8B409EF1DF0B3
:102D50008651380AD8B467EF1DF0C1EF1AF0079812
:102D6000079A04017A0E826FA4EC0AF00401780E2F
:102D7000826FA4EC0AF00401640E826FA4EC0AF0E6
:102D800081A8CAEF16F00401550E826FA4EC0AF078
:102D9000CFEF16F004014C0E826FA4EC0AF0AEECFB
:102DA0000AF0C1EF1AF00788079A04017A0E826FC1
:102DB000A4EC0AF00401410E826FA4EC0AF00401B5
:102DC000610E826FA4EC0AF0C0EF16F00798078A34
:102DD00004017A0E826FA4EC0AF00401420E826FA5
:102DE000A4EC0AF00401610E826FA4EC0AF0C0EFBB
:102DF00016F00101666704EF17F0676704EF17F03C
:102E0000686704EF17F069671CEF17F04F6710EF62
:102E100017F0506710EF17F0516710EF17F0526777
:102E20001CEF17F00101000E006F000E016F000E85
:102E3000026F000E036F12000101620E046F010E9B
:102E4000056F000E066F000E076F66C100F167C1C7
:102E500001F168C102F169C103F17DEC20F003BF0B
:102E6000A0EF17F00101000E046FA80E056F550EBC
:102E7000066F020E076F66C100F167C101F168C1FC
:102E800002F169C103F166C186F167C187F168C1CA
:102E900088F169C189F17DEC20F003BF59EF17F08B
:102EA0000101000E866FA80E876F550E886F020E07
:102EB000896F0E0EB0EC07F0E8CF18F10F0EB0ECF2
:102EC00007F0E8CF19F1100EB0EC07F0E8CF1AF1D7
:102ED000110EB0EC07F0E8CF1BF1C6EC1FF086C175
:102EE00004F187C105F188C106F189C107F17DECC4
:102EF00020F007828AEC1FF0C6EC1FF007928AECE4
:102F00001FF086C100F187C101F188C102F189C1BA
:102F100003F107928AEC1FF0CC0E046FE00E056FF0
:102F2000870E066F050E076F7DEC20F000C118F1CB
:102F300001C119F102C11AF103C11BF1D8EF17F059
:102F40000101800E006F1A0E016F060E026F000E57
:102F5000036F4FC104F150C105F151C106F152C1D7
:102F600007F17DEC20F003AFB9EF17F074EC21F01E
:102F700012000E0EB0EC07F0E8CF18F10F0EB0EC17
:102F800007F0E8CF19F1100EB0EC07F0E8CF1AF116
:102F9000110EB0EC07F0E8CF1BF14FC100F150C1AA
:102FA00001F151C102F152C103F107828AEC1FF015
:102FB00018C100F119C101F11AC102F11BC103F1DD
:102FC00012000401730E826FA4EC0AF004012C0EAF
:102FD000826FA4EC0AF0078462C166F163C167F1F5
:102FE00064C168F165C169F14BC14FF14CC150F149
:102FF0004DC151F14EC152F157C159F158C15AF169
:10300000079407EC18F0AEEC0AF0C1EF1AF066C1B5
:1030100000F167C101F168C102F169C103F1010169
:1030200017EC21F0FEEC1EF00401630E826FA4EC9D
:103030000AF004012C0E826FA4EC0AF04FC100F1DB
:1030400050C101F151C102F152C103F1010117EC6C
:1030500021F0FEEC1EF00401660E826FA4EC0AF073
:1030600004012C0E826FA4EC0AF074EC21F059C11B
:1030700000F15AC101F1010117EC21F0FEEC1EF044
:103080000401740E826FA4EC0AF012001082040195
:10309000530E826FA4EC0AF004012C0E826FA4EC94
:1030A0000AF083C32AF184C32BF185C32CF186C3B4
:1030B0002DF187C32EF188C32FF189C330F18AC364
:1030C00031F18BC332F18CC333F10101C2EC21F039
:1030D00039EC21F000C166F101C167F102C168F16C
:1030E00003C169F18EC32AF18FC32BF190C32CF178
:1030F00091C32DF192C32EF193C32FF194C330F1FC
:1031000095C331F196C332F197C333F10101C2EC9B
:1031100021F039EC21F000C14FF101C150F102C1A1
:1031200051F103C152F1B5EC21F099C32FF19AC3CB
:1031300030F19BC331F19CC332F19DC333F10101E6
:10314000C2EC21F039EC21F000C159F101C15AF172
:1031500007EC18F004012C0E826FA4EC0AF0B8EF13
:1031600018F08251520A03E10F82B8EF18F00F9263
:103170008251750A03E11084BFEF18F01094825158
:10318000550A03E11086C6EF18F01096078410B2B6
:1031900023EF19F010A40FEF19F0B6C166F1B7C113
:1031A00067F1B8C168F1B9C169F1BAC16AF1BBC1CF
:1031B0006BF1BCC16CF1BDC16DF1BEC16EF1BFC19F
:1031C0006FF1C0C170F1C1C171F1C2C172F1C3C16F
:1031D00073F1C4C174F1C5C175F1C6C176F1C7C13F
:1031E00077F1C8C178F1C9C179F1CAC17AF1CBC10F
:1031F0007BF1CCC17CF1CDC17DF1CEC17EF1CFC1DF
:103200007FF1D0C180F1D1C181F1D2C182F1D3C1AE
:1032100083F1D4C184F1D5C185F117EF19F062C1F2
:1032200066F163C167F164C168F165C169F14BC1C1
:103230004FF14CC150F14DC151F14EC152F157C146
:1032400059F158C15AF107940FA045EF19F0010147
:10325000926732EF19F0936732EF19F0946732EF0B
:1032600019F0956736EF19F045EF19F0F9EC16F003
:1032700092C104F193C105F194C106F195C107F122
:103280007DEC20F003BF89EF1AF0F9EC16F0010194
:10329000000E046F000E056F010E066F000E076F23
:1032A000ABEC20F010A45CEF19F00401750E826FF6
:1032B000A4EC0AF061EF19F00401720E826FA4EC25
:1032C0000AF004012C0E826FA4EC0AF017EC21F036
:1032D000296770EF19F00401200E826F73EF19F067
:1032E00004012D0E826FA4EC0AF030C182F40401B7
:1032F000300E8227A4EC0AF031C182F40401300EB2
:103300008227A4EC0AF004012E0E826FA4EC0AF0CE
:1033100032C182F40401300E8227A4EC0AF033C1DA
:1033200082F40401300E8227A4EC0AF004016D0E31
:10333000826FA4EC0AF004012C0E826FA4EC0AF058
:103340004FC100F150C101F151C102F152C103F16D
:10335000010117EC21F0FEEC1EF00401480E826F13
:10336000A4EC0AF004017A0E826FA4EC0AF00401C6
:103370002C0E826FA4EC0AF066C100F167C101F166
:1033800068C102F169C103F1010117EC21F0FEEC03
:103390001EF00401630E826FA4EC0AF004012C0EEF
:1033A000826FA4EC0AF066C100F167C101F168C147
:1033B00002F169C103F101010A0E046F000E056FED
:1033C000000E066F000E076F8CEC20F0000E046FED
:1033D000120E056F000E066F000E076FABEC20F0AB
:1033E00017EC21F02AC182F40401300E8227A4ECEC
:1033F0000AF02BC182F40401300E8227A4EC0AF0FB
:103400002CC182F40401300E8227A4EC0AF02DC1F5
:1034100082F40401300E8227A4EC0AF02EC182F45B
:103420000401300E8227A4EC0AF02FC182F40401BB
:10343000300E8227A4EC0AF030C182F40401300E71
:103440008227A4EC0AF004012E0E826FA4EC0AF08D
:1034500031C182F40401300E8227A4EC0AF032C19B
:1034600082F40401300E8227A4EC0AF033C182F406
:103470000401300E8227A4EC0AF00401730E826F5F
:10348000A4EC0AF004012C0E826FA4EC0AF074EC98
:1034900021F059C100F15AC101F1EBEC1BF00FB260
:1034A00055EF1AF00FA087EF1AF004012C0E826F6F
:1034B000A4EC0AF0200EF86EF76AF66A040109001F
:1034C000F5CF82F4A4EC0AF00900F5CF82F4A4EC65
:1034D0000AF00900F5CF82F4A4EC0AF00900F5CF58
:1034E00082F4A4EC0AF00900F5CF82F4A4EC0AF00F
:1034F0000900F5CF82F4A4EC0AF00900F5CF82F4BC
:10350000A4EC0AF00900F5CF82F4A4EC0AF0AEECCA
:103510000AF00F90C1EF1AF00401630E826FA4EC61
:103520000AF004012C0E826FA4EC0AF0C7EC1AF02A
:1035300004012C0E826FA4EC0AF03AEC1BF004019B
:103540002C0E826FA4EC0AF0B6EC1BF004012C0EDA
:10355000826FA4EC0AF00101F80E006FCD0E016F2E
:10356000660E026F030E036FDCEC1AF004012C0EE2
:10357000826FA4EC0AF0CCEC1BF0AEEC0AF0C1EFC9
:103580001AF00301C26B07901092D0EF1DF0D89093
:103590000E0EB0EC07F0E8CF00F10F0EB0EC07F024
:1035A000E8CF01F1100EB0EC07F0E8CF02F1110EF8
:1035B000B0EC07F0E8CF03F10101000E046F000E3C
:1035C000056F010E066F000E076FABEC20F017ECD5
:1035D00021F02AC182F40401300E8227A4EC0AF003
:1035E0002BC182F40401300E8227A4EC0AF02CC116
:1035F00082F40401300E8227A4EC0AF02DC182F47B
:103600000401300E8227A4EC0AF02EC182F40401DA
:10361000300E8227A4EC0AF02FC182F40401300E90
:103620008227A4EC0AF030C182F40401300E822714
:10363000A4EC0AF031C182F40401300E8227A4EC1C
:103640000AF004012E0E826FA4EC0AF032C182F45B
:103650000401300E8227A4EC0AF033C182F4040185
:10366000300E8227A4EC0AF004016D0E826FA4ECE8
:103670000AF01200120EB0EC07F0E8CF00F1130EC2
:10368000B0EC07F0E8CF01F1140EB0EC07F0E8CF92
:1036900002F1150EB0EC07F0E8CF03F101010A0EBC
:1036A000046F000E056F000E066F000E076F8CECA6
:1036B00020F0000E046F120E056F000E066F000E54
:1036C000076FABEC20F017EC21F02AC182F4040163
:1036D000300E8227A4EC0AF02BC182F40401300ED4
:1036E0008227A4EC0AF02CC182F40401300E822758
:1036F000A4EC0AF02DC182F40401300E8227A4EC60
:103700000AF02EC182F40401300E8227A4EC0AF0E4
:103710002FC182F40401300E8227A4EC0AF030C1DC
:1037200082F40401300E8227A4EC0AF004012E0E6C
:10373000826FA4EC0AF031C182F40401300E8227BA
:10374000A4EC0AF032C182F40401300E8227A4EC0A
:103750000AF033C182F40401300E8227A4EC0AF08F
:103760000401730E826FA4EC0AF012000A0EB0EC92
:1037700007F0E8CF00F10B0EB0EC07F0E8CF01F155
:103780000C0EB0EC07F0E8CF02F10D0EB0EC07F034
:10379000E8CF03F1EBEF1BF0060EB0EC07F0E8CF3B
:1037A00000F1070EB0EC07F0E8CF01F1080EB0EC25
:1037B00007F0E8CF02F1090EB0EC07F0E8CF03F113
:1037C000EBEF1BF0010174EC21F0078457C100F10D
:1037D00058C101F107940101E80E046F800E056FD6
:1037E000000E066F000E076F8CEC20F0000E046FC9
:1037F000040E056F000E066F000E076FABEC20F095
:10380000880E046F130E056F000E066F000E076F13
:103810007DEC20F00A0E046F000E056F000E066F9F
:10382000000E076FABEC20F017EC21F001012967C7
:103830001FEF1CF00401200E826F22EF1CF0040128
:103840002D0E826FA4EC0AF030C182F40401300E18
:103850008227A4EC0AF031C182F40401300E8227E1
:10386000A4EC0AF032C182F40401300E8227A4ECE9
:103870000AF004012E0E826FA4EC0AF033C182F428
:103880000401300E8227A4EC0AF00401430E826F7B
:10389000A4EC0AF0120087C32AF188C32BF189C374
:1038A0002CF18AC32DF18BC32EF18CC32FF18DC364
:1038B00030F18EC331F190C332F191C333F1010184
:1038C000296BC2EC21F039EC21F00101000E046FEC
:1038D000000E056F010E066F000E076F8CEC20F0D6
:1038E0000E0E0C6E00C10BF099EC07F00F0E0C6E73
:1038F00001C10BF099EC07F0100E0C6E02C10BF039
:1039000099EC07F0110E0C6E03C10BF099EC07F067
:1039100004017A0E826FA4EC0AF004012C0E826F6F
:10392000A4EC0AF00401350E826FA4EC0AF0040145
:103930002C0E826FA4EC0AF0C7EC1AF0CFEF16F051
:1039400087C32AF188C32BF189C32CF18AC32DF1D7
:103950008BC32EF18CC32FF18DC330F18EC331F1A7
:1039600090C332F191C333F10101296BC2EC21F014
:1039700039EC21F0880E046F130E056F000E066FF0
:10398000000E076F81EC20F0000E046F040E056F2F
:10399000000E066F000E076F8CEC20F00101E80EA0
:1039A000046F800E056F000E066F000E076FABEC04
:1039B00020F00A0E0C6E00C10BF099EC07F00B0E14
:1039C0000C6E01C10BF099EC07F00C0E0C6E02C1ED
:1039D0000BF099EC07F00D0E0C6E03C10BF099EC97
:1039E00007F004017A0E826FA4EC0AF004012C0E99
:1039F000826FA4EC0AF00401360E826FA4EC0AF088
:103A000004012C0E826FA4EC0AF0B6EC1BF0CFEF91
:103A100016F087C32AF188C32BF189C32CF18AC31E
:103A20002DF18BC32EF18CC32FF18DC330F18FC3D9
:103A300031F190C332F191C333F10101C2EC21F0B5
:103A400039EC21F0000E046F120E056F000E066FA8
:103A5000000E076F8CEC20F001010A0E046F000EBF
:103A6000056F000E066F000E076FABEC20F0120E14
:103A70000C6E00C10BF099EC07F0130E0C6E01C137
:103A80000BF099EC07F0140E0C6E02C10BF099ECE0
:103A900007F0150E0C6E03C10BF099EC07F0040152
:103AA0007A0E826FA4EC0AF004012C0E826FA4EC53
:103AB0000AF00401370E826FA4EC0AF004012C0E08
:103AC000826FA4EC0AF03AEC1BF0CFEF16F087C33C
:103AD0002AF188C32BF189C32CF18AC32DF18BC342
:103AE0002EF18CC32FF18DC330F18EC331F190C311
:103AF00032F191C333F10101296BC2EC21F039ECB1
:103B000021F0880E046F130E056F000E066F000E75
:103B1000076F81EC20F0000E046F040E056F000E9D
:103B2000066F000E076F8CEC20F00101E80E046FA9
:103B3000800E056F000E066F000E076FABEC20F0D5
:103B4000060E0C6E00C10BF099EC07F0070E0C6E20
:103B500001C10BF099EC07F0080E0C6E02C10BF0DE
:103B600099EC07F0090E0C6E03C10BF099EC07F00D
:103B700004017A0E826FA4EC0AF004012C0E826F0D
:103B8000A4EC0AF00401380E826FA4EC0AF00401E0
:103B90002C0E826FA4EC0AF0CCEC1BF0CFEF16F0E9
:103BA00081A88EEF1EF007A847EF1EF00101800EDE
:103BB000006F1A0E016F060E026F000E036F4BC1ED
:103BC00004F14CC105F14DC106F14EC107F17DEC88
:103BD00020F003BF8EEF1EF0F8EC1EF04BC100F199
:103BE0004CC101F14DC102F14EC103F107828AECD3
:103BF0001FF018C104F119C105F11AC106F11BC16A
:103C000007F1F80E006FCD0E016F660E026F030E06
:103C1000036F7DEC20F00E0E0C6E00C10BF099ECE2
:103C200007F00F0E0C6E01C10BF099EC07F0100EAF
:103C30000C6E02C10BF099EC07F0110E0C6E03C173
:103C40000BF099EC07F00784010174EC21F057C1E7
:103C500000F158C101F107940A0E0C6E00C10BF07F
:103C600099EC07F00B0E0C6E01C10BF099EC07F00C
:103C70000C0E0C6E02C10BF099EC07F00D0E0C6EE1
:103C800003C10BF099EC07F007988EEF1EF007AA1E
:103C90008EEF1EF00784010174EC21F057C100F192
:103CA00058C101F10794060E0C6E00C10BF099EC9F
:103CB00007F0070E0C6E01C10BF099EC07F0080E2F
:103CC0000C6E02C10BF099EC07F0090E0C6E03C1EB
:103CD0000BF099EC07F0078462C100F163C101F1B8
:103CE00064C102F165C103F10794120E0C6E00C1AC
:103CF0000BF099EC07F0130E0C6E01C10BF099EC70
:103D000007F0140E0C6E02C10BF099EC07F0150EC3
:103D10000C6E03C10BF099EC07F0079A0401805177
:103D200081197F0B0BE09EA809D014EE00F08151A1
:103D30007F0BE126E750812B0F01AD6E0501295164
:103D4000010A13E081AAB5EF1EF005012951000A0E
:103D50000AE00FB8B5EF1EF005012A67B5EF1EF0B7
:103D60000FB8B5EF1EF0B2EF27F081B8CAEF1EF022
:103D7000DDEC23F005012951020A02E0CAEF1EF032
:103D8000562FCAEF1EF055C556F50501010E2A6FD4
:103D90003C0E2B6F0DEF0AF018C100F119C101F1B3
:103DA0001AC102F11BC103F1000E046F000E056F72
:103DB000010E066F000E076FABEC20F029A1F7EFA4
:103DC0001EF02051D8B4F7EF1EF018C100F119C150
:103DD00001F11AC102F11BC103F1000E046F000EC4
:103DE000056F0A0E066F000E076FABEC20F0120095
:103DF0000101186B196B1A6B1B6B12002AC182F43C
:103E00000401300E8227A4EC0AF02BC182F40401D5
:103E1000300E8227A4EC0AF02CC182F40401300E8B
:103E20008227A4EC0AF02DC182F40401300E82270F
:103E3000A4EC0AF02EC182F40401300E8227A4EC17
:103E40000AF02FC182F40401300E8227A4EC0AF09C
:103E500030C182F40401300E8227A4EC0AF031C193
:103E600082F40401300E8227A4EC0AF032C182F4FD
:103E70000401300E8227A4EC0AF033C182F404015D
:103E8000300E8227A4EC0AF012002FC182F4040144
:103E9000300E8227A4EC0AF030C182F40401300E07
:103EA0008227A4EC0AF031C182F40401300E82278B
:103EB000A4EC0AF032C182F40401300E8227A4EC93
:103EC0000AF033C182F40401300E8227A4EC0AF018
:103ED0001200060E116E060E126E060E136E112ED5
:103EE0006FEF1FF0122E6FEF1FF0132E6FEF1FF00A
:103EF0008B84020E116E020E126E020E136E112EC4
:103F00007FEF1FF0122E7FEF1FF0132E7FEF1FF0B9
:103F10008B9412000101005305E1015303E10253A8
:103F200001E1002B4DEC20F074EC21F03951006FD1
:103F30003A51016F420E046F4B0E056F000E066F73
:103F4000000E076F8CEC20F000C104F101C105F1F7
:103F500002C106F103C107F118C100F119C101F155
:103F60001AC102F11BC103F107B2BBEF1FF081ECD4
:103F700020F0BDEF1FF07DEC20F000C118F101C171
:103F800019F102C11AF103C11BF1120074EC21F006
:103F900059C100F15AC101F1060EB0EC07F0E8CFAB
:103FA00004F1070EB0EC07F0E8CF05F1080EB0EC15
:103FB00007F0E8CF06F1090EB0EC07F0E8CF07F103
:103FC0007DEC20F000C124F101C125F102C126F1F0
:103FD00003C127F1290E046F000E056F000E066F56
:103FE000000E076F8CEC20F0EE0E046F430E056F91
:103FF000000E066F000E076F81EC20F024C104F163
:1040000025C105F126C106F127C107F18CEC20F08E
:1040100000C11CF101C11DF102C11EF103C11FF15C
:10402000120EB0EC07F0E8CF04F1130EB0EC07F07D
:10403000E8CF05F1140EB0EC07F0E8CF06F1150E4D
:10404000B0EC07F0E8CF07F10D0E006F000E016F26
:10405000000E026F000E036F8CEC20F0180E046F40
:10406000000E056F000E066F000E076FABEC20F020
:104070001CC104F11DC105F11EC106F11FC107F1EC
:1040800081EC20F06A0E046F2A0E056F000E066F99
:10409000000E076F7DEC20F01200BF0EFA6E200EAE
:1040A0003A6F396BD8900037013702370337D8B0F1
:1040B0005EEF20F03A2F53EF20F039073A07035311
:1040C000D8B412000331070B80093F6F03390F0B7F
:1040D000010F396F80EC5FF0406F390580EC5FF0C5
:1040E000405D405F396B3F33D8B0392739333FA942
:1040F00073EF20F040513927120099EC21F0D8B02D
:10410000120003510719346F5CEC21F0D89007516D
:10411000031934AF800F1200346B80EC21F0D8A06B
:1041200096EC21F0D8B012006BEC21F074EC21F089
:104130001F0E366FACEC21F00B35D8B05CEC21F0E3
:10414000D8A00335D8B01200362F9AEF20F034B142
:1041500083EC21F01200346B045105110611071194
:104160000008D8A080EC21F0D8A096EC21F0D8B0BF
:104170001200086B096B0A6B0B6BACEC21F01F0E85
:10418000366FACEC21F007510B5DD8A4D4EF20F0D2
:1041900006510A5DD8A4D4EF20F00551095DD8A4DA
:1041A000D4EF20F00451085DD8A0E7EF20F00451CF
:1041B000085F0551D8A0053D095F0651D8A0063D0E
:1041C0000A5F0751D8A0073D0B5FD8900081362FBA
:1041D000C1EF20F034B183EC21F0346B80EC21F09E
:1041E000D890B0EC21F007510B5DD8A404EF21F07A
:1041F00006510A5DD8A404EF21F00551095DD8A449
:1042000004EF21F00451085DD8A013EF21F0003F26
:1042100013EF21F0013F13EF21F0023F13EF21F0E4
:10422000032BD8B4120034B183EC21F01200010149
:10423000346B80EC21F0D8B01200B5EC21F0200EE8
:10424000366F003701370237033711EE33F00A0EAD
:10425000376FE7360A0EE75CD8B0E76EE552372FC6
:1042600029EF21F0362F21EF21F034B12981D890A8
:10427000120001010A0E346F200E366F11EE29F084
:104280003451376F0A0ED890E652D8B0E726E7329D
:10429000372F44EF21F00333023301330033362F3D
:1042A0003EEF21F0E750FF0FD8A00335D8B0120041
:1042B00029B183EC21F01200045100270551D8B038
:1042C000053D01270651D8B0063D02270751D8B059
:1042D000073D032712000051086F0151096F025179
:1042E0000A6F03510B6F12000101006B016B026B2F
:1042F000036B12000101046B056B066B076B120068
:104300000335D8A012000351800B001F011F021FAC
:10431000031F003F93EF21F0013F93EF21F0023F95
:1043200093EF21F0032B342B032512000735D8A07F
:1043300012000751800B041F051F061F071F043FB3
:10434000A9EF21F0053FA9EF21F0063FA9EF21F0E9
:10435000072B342B072512000037013702370337AC
:10436000083709370A370B3712000101296B2A6B0E
:104370002B6B2C6B2D6B2E6B2F6B306B316B326B71
:10438000336B120001012A510F0B2A6F2B510F0BB7
:104390002B6F2C510F0B2C6F2D510F0B2D6F2E519E
:1043A0000F0B2E6F2F510F0B2F6F30510F0B306FE4
:1043B00031510F0B316F32510F0B326F33510F0BE5
:1043C000336F12008A94000EC76E200EC66E9E9642
:1043D000C69EC50EC96EFF0E9EB602D0E82EFCD753
:1043E0009E96C69E000EC96EFF0E9EB602D0E82EA7
:1043F000FCD7C9CF00F69E96C69E000EC96EFF0E72
:104400009EB602D0E82EFCD7C9CF01F68A841200EE
:10441000000EC76E200EC66E8A949E96C69EC80E6B
:10442000C96EFF0E9EB602D0E82EFCD79E96C69EA1
:10443000000EC96EFF0E9EB602D0E82EFCD7C9CF83
:1044400002F69E96C69E000EC96EFF0E9EB602D064
:10445000E82EFCD7C9CF03F68A848A949E96C69E1E
:10446000CA0EC96EFF0E9EB602D0E82EFCD79E96ED
:10447000C69E000EC96EFF0E9EB602D0E82EFCD777
:10448000C9CF04F69E96C69E000EC96EFF0E9EB65C
:1044900002D0E82EFCD7C9CF05F68A848A949E966E
:1044A000C69ECC0EC96EFF0E9EB602D0E82EFCD77B
:1044B0009E96C69E000EC96EFF0E9EB602D0E82ED6
:1044C000FCD7C9CF06F69E96C69E000EC96EFF0E9B
:1044D0009EB602D0E82EFCD7C9CF07F68A84120018
:1044E000000EC76E200EC66E8A949E96C69EE80E7B
:1044F000C96EFF0E9EB602D0E82EFCD79E96C69ED1
:10450000000EC96EFF0E9EB602D0E82EFCD7C9CFB2
:1045100008F69E96C69E000EC96EFF0E9EB602D08D
:10452000E82EFCD7C9CF09F68A848A949E96C69E47
:10453000EA0EC96EFF0E9EB602D0E82EFCD79E96FC
:10454000C69E000EC96EFF0E9EB602D0E82EFCD7A6
:10455000C9CF0AF69E96C69E000EC96EFF0E9EB685
:1045600002D0E82EFCD7C9CF0BF68A848A949E9697
:10457000C69EEC0EC96EFF0E9EB602D0E82EFCD78A
:104580009E96C69E000EC96EFF0E9EB602D0E82E05
:10459000FCD7C9CF0CF69E96C69E000EC96EFF0EC4
:1045A0009EB602D0E82EFCD7C9CF0DF68A84120041
:1045B000000EC76E200EC66E8A949E96C69E240E6E
:1045C000C96EFF0E9EB602D0E82EFCD79E96C69E00
:1045D000E40EC96EFF0E9EB602D0E82EFCD78A8488
:1045E0008A949E96C69E200EC96EFF0E9EB602D07D
:1045F000E82EFCD79E96C69E5F0EC96EFF0E9EB635
:1046000002D0E82EFCD78A848A949E96C69E210EFC
:10461000C96EFF0E9EB602D0E82EFCD79E96C69EAF
:10462000C00EC96EFF0E9EB602D0E82EFCD78A845B
:104630008A949E96C69E260EC96EFF0E9EB602D026
:10464000E82EFCD79E96C69E000EC96EFF0E9EB643
:1046500002D0E82EFCD78A8412008984000EC76E2F
:10466000220EC66E9E96C69E000EC96EFF0E9EB6A8
:1046700002D0E82EFCD79E96C69E000EC96EFF0E95
:104680009EB602D0E82EFCD7C9CFA5F59E96C69E51
:10469000000EC96EFF0E9EB602D0E82EFCD7C9CF21
:1046A000A6F59E96C69E000EC96EFF0E9EB602D05F
:1046B000E82EFCD7C9CFA7F59E96C69E000EC96E00
:1046C000FF0E9EB602D0E82EFCD7C9CFA8F59E9665
:1046D000C69E000EC96EFF0E9EB602D0E82EFCD715
:1046E000C9CFA9F59E96C69E000EC96EFF0E9EB656
:1046F00002D0E82EFCD7C9CFAAF59E96C69E000E22
:10470000C96EFF0E9EB602D0E82EFCD7C9CFABF51E
:104710008994E0EC25F012008984000EC76E220E09
:10472000C66E9E96C69E800EC96EFF0E9EB602D0C5
:10473000E82EFCD79E96C69EA5C5C9FFFF0E9EB665
:1047400002D0E82EFCD79E96C69EA6C5C9FFFF0ED6
:104750009EB602D0E82EFCD79E96C69EA7C5C9FF7E
:10476000FF0E9EB602D0E82EFCD79E96C69EA8C528
:10477000C9FFFF0E9EB602D0E82EFCD79E96C69EBD
:10478000A9C5C9FFFF0E9EB602D0E82EFCD79E96A3
:10479000C69EAAC5C9FFFF0E9EB602D0E82EFCD762
:1047A0009E96C69EABC5C9FFFF0E9EB602D0E82EF0
:1047B000FCD78994E0EC25F012008984000EC76EC6
:1047C000220EC66E9E96C69E070EC96EFF0E9EB640
:1047D00002D0E82EFCD79E96C69E000EC96EFF0E34
:1047E0009EB602D0E82EFCD7C9CFA5F59E96C69EF0
:1047F000000EC96EFF0E9EB602D0E82EFCD7C9CFC0
:10480000A6F59E96C69E000EC96EFF0E9EB602D0FD
:10481000E82EFCD7C9CFA7F59E96C69E000EC96E9E
:10482000FF0E9EB602D0E82EFCD7C9CFA8F589941A
:10483000E0EC25F08984000EC76E220EC66E9E96AF
:10484000C69E0F0EC96EFF0E9EB602D0E82EFCD794
:104850009E96C69E000EC96EFF0E9EB602D0E82E32
:10486000FCD7C9CFADF58994E0EC25F0120089841E
:10487000000EC76E220EC66E9E96C69E870EC96E2D
:10488000FF0E9EB602D0E82EFCD79E96C69EA5C50A
:10489000C9FFFF0E9EB602D0E82EFCD79E96C69E9C
:1048A000A6C5C9FFFF0E9EB602D0E82EFCD79E9685
:1048B000C69EA7C5C9FFFF0E9EB602D0E82EFCD744
:1048C0009E96C69EA8C5C9FFFF0E9EB602D0E82ED2
:1048D000FCD78994E0EC25F089849E96C69E8F0EC5
:1048E000C96EFF0E9EB602D0E82EFCD79E96C69EDD
:1048F000ADC5C9FFFF0E9EB602D0E82EFCD7899445
:10490000E0EC25F012008984000EC76E220EC66E00
:104910009E96C69E870EC96EFF0E9EB602D0E82EEA
:10492000FCD79E96C69E000EC96EFF0E9EB602D0A4
:10493000E82EFCD79E96C69E800EC96EFF0E9EB6D0
:1049400002D0E82EFCD79E96C69E800EC96EFF0E42
:104950009EB602D0E82EFCD79E96C69E800EC96EEB
:10496000FF0E9EB602D0E82EFCD78994E0EC25F02D
:1049700089849E96C69E8F0EC96EFF0E9EB602D08B
:10498000E82EFCD79E96C69E010EC96EFF0E9EB6FF
:1049900002D0E82EFCD78994E0EC25F0120089843F
:1049A000000EC76E220EC66E9E96C69E870EC96EFC
:1049B000FF0E9EB602D0E82EFCD79E96C69E000E35
:1049C000C96EFF0E9EB602D0E82EFCD79E96C69EFC
:1049D000000EC96EFF0E9EB602D0E82EFCD79E9642
:1049E000C69E800EC96EFF0E9EB602D0E82EFCD782
:1049F0009E96C69E800EC96EFF0E9EB602D0E82E11
:104A0000FCD78994E0EC25F089849E96C69E8F0E93
:104A1000C96EFF0E9EB602D0E82EFCD79E96C69EAB
:104A2000010EC96EFF0E9EB602D0E82EFCD7899407
:104A3000E0EC25F012008984000EC76E220EC66ECF
:104A40009E96C69E8F0EC96EFF0E9EB602D0E82EB1
:104A5000FCD7E0EC25F09E96C69E810EC96EFF0E37
:104A60009EB602D0E82EFCD78994E0EC25F089842C
:104A7000000EC76E220EC66E9E96C69E8F0EC96E23
:104A8000FF0E9EB602D0E82EFCD7E0EC25F09E96F5
:104A9000C69E010EC96EFF0E9EB602D0E82EFCD750
:104AA0008994E0EC25F089849E96C69E910EC96E8D
:104AB000FF0E9EB602D0E82EFCD7E0EC25F09E96C5
:104AC000C69EA50EC96EFF0E9EB602D0E82EFCD77C
:104AD0008994E0EC25F012008984000EC76E220E46
:104AE000C66E9E96C69E8F0EC96EFF0E9EB602D0F3
:104AF000E82EFCD7E0EC25F09E96C69E810EC96E8E
:104B0000FF0E9EB602D0E82EFCD78994E0EC25F08B
:104B100012008984000EC76E220EC66E9E96C69E37
:104B20008F0EC96EFF0E9EB602D0E82EFCD7E0ECC9
:104B300025F09E96C69E010EC96EFF0E9EB602D04F
:104B4000E82EFCD78994E0EC25F012008984000E51
:104B5000C76E220EC66E9E96C69E910EC96EFF0E41
:104B60009EB602D0E82EFCD7E0EC25F09E96C69EBD
:104B7000A50EC96EFF0E9EB602D0E82EFCD7899412
:104B8000E0EC25F012008984000EC76E220EC66E7E
:104B90009E96C69E910EC96EFF0E9EB602D0E82E5E
:104BA000FCD7E0EC25F09E96C69E000EC96EFF0E67
:104BB0009EB602D0E82EFCD78994E0EC25F01200D6
:104BC000050EE82EFED71200200EC66E0501256BDD
:104BD000266B276B286B899A400EC76E200EC66E17
:104BE0009E96C69E030EC96EFF0E9EB602D0E82E9C
:104BF000FCD79E96C69E27C5C9FFFF0E9EB602D063
:104C0000E82EFCD79E96C69E26C5C9FFFF0E9EB60F
:104C100002D0E82EFCD79E96C69E25C5C9FFFF0E82
:104C20009EB602D0E82EFCD79E96C69EC952FF0EB5
:104C30009EB602D0E82EFCD7898AC950FF0A02E14D
:104C40002BEF26F0100E2527E86A2623E86A272393
:104C500027A9EBEF25F0220EC66E1200899A400EAE
:104C6000C76E200EC66E9E96C69E060EC96EFF0EBD
:104C70009EB602D0E82EFCD7898A899A9E96C69E57
:104C8000C70EC96EFF0E9EB602D0E82EFCD7898AE9
:104C9000899A9E96C69E050EC96EFF0E9EB602D0DC
:104CA000E82EFCD79E96C69EC952FF0E9EB602D035
:104CB000E82EFCD7C9B052EF26F0898A0501256B92
:104CC000266B276B286B12000501FE0E2D6F050168
:104CD000000E2D6F2DEC23F0A5C52EF5A6C52FF5E2
:104CE000A7C530F5A8C531F5A9C532F5AAC533F574
:104CF000ABC534F50784B6C166F1B7C167F1B8C179
:104D000068F1B9C169F14BC14FF14CC150F14DC1CE
:104D100051F14EC152F157C159F158C15AF107949E
:104D2000F9EC16F000C135F501C136F502C137F5D1
:104D300003C138F505015767A5EF26F05867A5EFC1
:104D400026F05967A5EF26F05A67A9EF26F0B7EFCE
:104D500026F057C504F158C505F159C506F15AC5E5
:104D600007F101017DEC20F003BF25EF27F059C1C9
:104D700039F55AC13AF5AFC53BF5B0C53CF505016B
:104D8000100E2C6F899A400EC76E200EC66E9E962E
:104D9000C69E060EC96EFF0E9EB602D0E82EFCD748
:104DA000898A899A9E96C69E020EC96EFF0E9EB68D
:104DB00002D0E82EFCD79E96C69E27C5C9FFFF0EDF
:104DC0009EB602D0E82EFCD79E96C69E26C5C9FF89
:104DD000FF0E9EB602D0E82EFCD79E96C69E25C535
:104DE000C9FFFF0E9EB602D0E82EFCD725EE2DF0AF
:104DF0002C2F02D007EF27F09E96C69EDECFC9FF6C
:104E0000FF0E9EB602D0E82EFCD7F8EF26F0898A76
:104E1000899A9E96C69E050EC96EFF0E9EB602D05A
:104E2000E82EFCD79E96C69EC952FF0E9EB602D0B3
:104E3000E82EFCD7C9B012EF27F0898A0501100EC1
:104E40002527E86A2623E86A2723120021C500F1F6
:104E500022C501F123C502F124C503F1899A400E50
:104E6000C76E200EC66E9E96C69E0B0EC96EFF0EB6
:104E70009EB602D0E82EFCD79E96C69E02C1C9FF00
:104E8000FF0E9EB602D0E82EFCD79E96C69E01C1AC
:104E9000C9FFFF0E9EB602D0E82EFCD79E96C69E96
:104EA00000C1C9FFFF0E9EB602D0E82EFCD79E9629
:104EB000C69EC952FF0E9EB602D0E82EFCD725EE44
:104EC0002DF00501100E2C6F9E96C69EC952FF0E46
:104ED0009EB602D0E82EFCD7C9CFDEFF2C2F64EFA0
:104EE00027F0898A1200899A400EC76E200EC66E7E
:104EF0009E96C69E900EC96EFF0E9EB602D0E82EFC
:104F0000FCD79E96C69E000EC96EFF0E9EB602D0BE
:104F1000E82EFCD79E96C69E000EC96EFF0E9EB66A
:104F200002D0E82EFCD79E96C69E000EC96EFF0EDC
:104F30009EB602D0E82EFCD79E96C69EC952FF0EA2
:104F40009EB602D0E82EFCD7C9CF2DF59E96C69E00
:104F5000C952FF0E9EB602D0E82EFCD7C9CF2EF55F
:104F6000898A1200DDEC23F0F29CF29E8B94899CDE
:104F7000C69AC2908A848A96898A9482948C720E88
:104F8000D36ED3A4FED789968A909390FF0EE8CF74
:104F900000F0E82EFED7002EFCD78150F294F29A52
:104FA0009E909D909E929D92F298F292F290F2863F
:064FB000F28E0300FF0079
:10BF0000E844F926000C160C2B0C3F0C520C640C68
:10BF1000760C860C960CA50CB30CC10CCF0CDC0C6B
:06BF2000E80CF40C000C1B
:00000001FF
